:020000040000FA
:060000000219FD02031CC1
:03000B0002008D63
:03001300020537AC
:03001B0002009050
:03002B000202D1FD
:03005B0002054655
:030073000203097C
:100080000406080C10182030406080A0C0054032E3
:10009000C2AFC2A853E6EFC28E856B8BC0D0D2D35D
:1000A000C0E0C0F0C2CAA8CCA9CDD2CAD2AF758A6E
:1000B00000C3E8956CF8E9956DF9C3E913F9E81305
:1000C000F8E5666007C3E913F9E813F8E97025E875
:1000D000956E4020956E501CE582B410177C007B15
:1000E000007A007908900000A86AE5667004C3E809
:1000F00013F801FD900000D2A8D2AA61E7E0FDC389
:100100009CC39840EF98EB33FB0582E0FCC39DC392
:100110009840E198EB33FB0582E0FDC39CC3984017
:10012000D398EB33FB0582E0FCC39DC39840C59890
:10013000EB33FB0582E0FDC39CC39840B798EB33DB
:10014000FB0582E0FCC39DC39840A998EB33FB05F7
:1001500082E0FDC39CC398409B98EB33FB0582E093
:10016000FCC39DC398408D98EB33FB0582217890AA
:100170000000D2A8D2AA61E7E0FDC39CC39840EF7B
:1001800098EA33FA0582E0FCC39DC39840E198EAFF
:1001900033FA0582E0FDC39CC39840D398EA33FA52
:1001A0000582E0FCC39DC39840C598EA33FA0582F6
:1001B000E0FDC39CC39840B798EA33FA0582E0FC9F
:1001C000C39DC39840A998EA33FA0582E0FDC39C19
:1001D000C398409B98EA33FA0582E0FCC39DC3981C
:1001E000408D98EA33FA0582EBC46B6A54F0F9EA61
:1001F000C454F0C3996009900000D2A8D2AA61E764
:10020000EBF4C454F0F9EAF4C4540F49FAEBF4C423
:10021000540FFBC3EAF99460FAEB9400FB5020C33F
:10022000E97B007A0079006016C3135006F9C39584
:1002300052600AE9F5527553007900800205533087
:100240003A27C3EA94D0F8EB9407F9400BE8FAE9AF
:10025000FB203509D235415D303502C235203902E7
:10026000B235C3EA33FAEB33FBEB2B3B3BF9C3EB81
:1002700013FBEA13FAEA29FAEB3400FB30E3047AC1
:10028000FF7BFFE5255403601B202A18E55D33F949
:10029000EB7007C3E99A4002E9FAE53CC4332AFA55
:1002A000EB3400FBC3EA33C4540FF8EB33C454F00F
:1002B00048F87005EA60027801900000D2A8D2AA3E
:1002C000E5226002152281D4900000D2A8D2AA6152
:1002D000E7C0D0C0E0C2CF0541E5666009E56560D2
:1002E000057565006104756501E52360021523C38A
:1002F000E55460057555006104E5552401F5555038
:10030000037555FFD0E0D0D032C2AF53E67F75926F
:10031000FA7593FFC22053917FD2AF32C0E0E58AD5
:10032000303408856B8BF0A3D0E032D0E0C2AF53FD
:10033000E6EFC0D0C0E0C0F0D2D3D2AF5388EFA870
:100340008AA98CAA40308D010A758A00758C0075C7
:100350004000438810E566700AC3E833F8E933F9D2
:10036000EA33FA30331FE8C4540FFAE9C454F04AB0
:10037000FAC3132AFAC3E833F8E933F9E82AFAE9A9
:100380003406FB61D830320FC3E833E933FAE82A88
:10039000FAE93400FB61D8303115E875F056A4AAAB
:1003A000F0E975F056A42AFAC5F03400FB61D8C311
:1003B000EA13FAE913F9E813F8E875F056A4AAF07D
:1003C000E975F056A42AFAC5F03400C313FBEA130A
:1003D000FAC3EB13FBEA13FAC3EB94125009C3EA16
:1003E0009434EB940750160522E52270021522C3BF
:1003F000E52294325002A12A755400A12DE5226015
:100400000215223036067C007D088117AC31AD32F2
:10041000303A04AC33AD34C3EA9CFAEB9DFB92084E
:10042000AE60AF61303A425007203509D235813590
:10043000303502C235303504AE62AF63203902B2C6
:1004400035C3EA33FAEB33FBA208500AEAF424017D
:10045000FAEBF43400FBC3EA9450FAEB9400FB503F
:100460001478007A007B008175A208500878007A21
:10047000007B0081D4E5255403601B202A18E55D2C
:1004800033F9EB7007C3E99A4002E9FAE53CC4335B
:100490002AFAEB3400FBEA8EF0A4F9AAF0EB8EF016
:1004A000A42AFAC5F03400FBC3EB13FDEA13F8C32A
:1004B000ED13FDE813F80FEF146004C3E833F8C33D
:1004C000E933EA33FAEB33FBDFEDEB30E30678FF99
:1004D0007AFF7B078854D230E86003755500C3E586
:1004E0005BFC955C4002AC5CC3EC95545008EC7529
:1004F000F008A4FAABF0EAF4F8EBF45407F98856E4
:10050000895775230AE55A30E210D0F0D0E0D0D0F8
:1005100053F7DF43F74043E61032D0F0D0E0D0D0BD
:1005200053D8FE43DA0143E6103275230AD0F0D0E7
:10053000E0D0D043E61032C2AAD28EC2CA85CC6CBB
:1005400085CD6DD2CA32C2AFC0D0C0E0D2D38556FD
:10055000FB8557FC85575A53F7BF53DAFED2A830B4
:100560003402D2AA53E6EF53F7DF53D8FED0E0D0DF
:10057000D0D2AF327901801479038010790A800CCF
:10058000791E80087964800479C880007817E4D5E2
:10059000E0FDD8FAD9F62278FF20282879A1E76073
:1005A00023E548601F74FF8548F084853FF03029BB
:1005B0000375F005A4F8C5F0600278FFC3E8955D07
:1005C0005002A85D885C22C3E54794A0E5489400EA
:1005D000E55C500314A1D8046002F55C2275E89034
:1005E00022055EC3E55E9408405330EDF4A8BDA932
:1005F000BE755E00E9FA79A0E76041EA7006E55F42
:100600006018800CC3E8955F600EE55F5005600AD6
:100610001480070460FA8002E55FF55FC3956940C6
:100620001B755BC0C394044013755B80C394044086
:100630000B755B40C394044003755B0022E55B24AB
:1006400010500274FFF55B22743279A687F0A4C5BE
:10065000F0A2F733F55D227547007548F022C2AF6E
:10066000C2CAA8CCA9CDAA4130CF010AD2CAD2AF02
:10067000C3EA13FAE913F9E813F8AB42AC43884232
:100680008943C3E89BF8E99C20280A547FF9302C61
:1006900002E17CC1D5AD448A44F9EA9D547FFA60F9
:1006A0000678FF79FFC1BAAE45AF468B458C46A8A8
:1006B00042A943C3E89EF8E99FF9C3E54813FBE567
:1006C0004713FAE82AF547E93BF54850067547FF16
:1006D0007548FFE122AA47AB48AC47AD487E047F8E
:1006E00002C3EB9404400D1E1FC3EB940840052089
:1006F00029021E1FC3ED13FDEC13FCDEF7C3EA9CB9
:10070000FAEB9DFBEF6009C3E913F9E813F8DFF793
:10071000EA28FAEB39FB8A478B4850067BFF8B4768
:100720008B48C3EB94025002D22C3028047F03E1A3
:100730004D7892E6FFC3E53D948240110FC3E53D3D
:1007400094A040010FC3EF940640027F057E02E5AE
:1007500048C4540FF9E548C454F0F8E547C4540FB1
:1007600028F8C3E89EFAE99400FB4009C3EA940123
:10077000EB940050047A01E4FB0207C8AA47AB4897
:10078000EBC4FEEAC4540F4EFCC3EA9CFAEB94009F
:10079000FBC3E813C313F8EA28FAEB3400FB8A47DB
:1007A0008B48C3EB94024002C22C7802EBC4FE7B60
:1007B00000EAC4540F4EFAC3EA98FA4005C3940104
:1007C00050027A017892E6FF302002E1C8854E920D
:1007D000854F93D22043E680C3E49AF8E49BF9C3A3
:1007E000E833F8E933F9302C0302085DE8FAE9FB55
:1007F000D3E913FDE813FC884E894FC3EF940360DF
:1008000038EF20E00CE82CF8E93DF9ECFAEDFB803C
:1008100013E828F8E939F9C3E82401F8E93400F9C4
:100820007AFF7BFFC3EF9403400F8A508B51884AB5
:10083000894B8C4C8D4D020892885089518A4A8B85
:100840004B8C4C8D4D3028127550F07551FF754C06
:10085000F0754DFF754EF0754FFF020892E8FAD320
:10086000E813FC884EC3EF94036021EF20E007E813
:100870002CF8ECFA017DE8282401F87AFFC3EF9404
:100880000340098A50884A8C4C02089288508A4A50
:100890008C4C3020020192753A02D22043E680E56A
:1008A000255403602DA847A948C3E913F9E813F8B4
:1008B000302804E92440F9C2AF53E67F759100C3A4
:1008C000E498F594E499F595759104D22043E68077
:1008D000D2AF22D221754900752000302B0375203C
:1008E0004001F1D221754900752040302B0375205D
:1008F0000078017901202C20E52554036002C221F3
:100900007914E548C313700104F8C39414400278C5
:1009100014302804781B791BC3E833F8C3E933F992
:10092000202010E549600C302803D53A04D222215A
:10093000A4119A0549E59B5440B52002218E302828
:100940000908C3E899400118212020210A08C3E8BA
:1009500099400201F12120C22153E67F75910030B8
:100960002C117594007595F0759104D22043E680A2
:100970000208F1E5487EFFC3334009C3334005C395
:10098000334001FEC3E49E759400F5952168C3E5EC
:10099000399401500201F130210201F1D80221A263
:1009A0002120C222C2AF53E67F7591008550948505
:1009B0005195759104854A92854B93D22043E680E8
:1009C000D2AFE52554036007202902053980103095
:1009D000220D202B0A2021071581158102141222D5
:1009E00078003021027801E53D75F007A4F9E5F0C3
:1009F00028F5F0E9A2F013A2F113A2F213F53DC31A
:100A000094785003753D78C3E53D953E400CC28710
:100A1000C291C29375D4FF75D50F302002411A855B
:100A20004C92854D93D22043E68022203817C2AFE6
:100A3000C291C286D287D29375D4FF75D50BD2AF3F
:100A4000759F42614FC2AFC291C292D293D2877555
:100A5000D4BF75D50FD2AF759F42614F203817C2F2
:100A6000AFC293D29175D4FF75D50EC286D287D20C
:100A7000AF759F52614FC2AFC287D29175D4FF75D7
:100A8000D50EC292D293D2AF759F32614F203817E4
:100A9000C2AFC287C292D293D29175D4FF75D50EE0
:100AA000D2AF759F32614FC2AFC293C286D287D296
:100AB0009175D4FF75D50ED2AF759F52614F203816
:100AC00017C2AFC291D28775D4BF75D50FC292D26B
:100AD00093D2AF759F428077C2AFC291D29375D443
:100AE000FF75D50BC286D287D2AF759F428060203A
:100AF0003817C2AFC293C290D291D28775D4BF7556
:100B0000D50FD2AF759F528046C2AFC287C290D276
:100B100091D29375D4FF75D50BD2AF759F32802FCC
:100B2000203817C2AFC287D29375D4FF75D50BC2D8
:100B300090D291D2AF759F328015C2AFC293D28747
:100B400075D4BF75D50FC290D291D2AF759F522286
:100B50007A147B7880127A107B8C800C7A0D7BB4AF
:100B600080067A0B7BC88000E564D5E0012279021B
:100B7000E4C291D5E0FDD290D291D5E0FDC291D5ED
:100B8000E0FDC290D291D5E0FDE920E004D286D20A
:100B90008730E004D292D293E564D5E0FDE920E00D
:100BA00002C28730E002C2937496D5E0FDD9C1EA53
:100BB000F8D5E0FDD8FBDBB0C29122C287C291C25A
:100BC00093C287C291C29375D4FF75D50F227880E6
:100BD00076FF0876FF0876FF0876FF0876FF08762E
:100BE000FF0876090876FF087601788C760108768A
:100BF000FF0876FF0876FF0876FF0876FF08760381
:100C00000876FF0876FF0876FF0876250876D00874
:100C100076280876500876040876FF08760208766B
:100C2000FF08767A0876FF0876070876010876FFCF
:100C30000876FF08760008760022FA75F00CA4AB5F
:100C4000F0EAC333F8740133F9E8C333F8E933F950
:100C5000E8C32BF8E93400F9E8C333F8E933F922A3
:100C60007888E6C39403D23A5002C23AC238E630DA
:100C7000E102D238A23892397886E6149000809347
:100C800078A6F67886E6F53FC394025003753F02D6
:100C9000789CE6753EFFB40203753EA0B40303756D
:100CA0003E8278A0E6F8600674282409D8FCF5692D
:100CB0007896E6913A88318932789EE6913A88337F
:100CC00089347897E6913A8835893671BB22303677
:100CD000117A007B007CFF7D007E00B1348B618A3D
:100CE0006022303A227896E6FA7B00789EE6FC7D18
:100CF00000C3EA33FAEB33FBC3EC33FCED33FD7E88
:100D00000AB1348B638A627896303A02789EE6FAAA
:100D10007B007897E6FC7D007E00303A10C3EA3312
:100D2000FAEB33FBC3EC33FCED33FD7E0AB1348BBD
:100D3000618A6022C3EC9EFCED9400FDC3EC9AFC3A
:100D4000ED9BFDC3EC9423ED940050047C237D00C7
:100D5000C3EC94FFED940140047CFF7D017BFF0B0D
:100D60007A000AEA7009C3EC33FCED33FDA15FECB5
:100D70008AF0A4AEF0ED8AF0A42E947C40E4EAF46C
:100D800060DD22D23691CE1205801205807A007B7A
:100D9000007C10120578E5542AFA74003BFBDCF362
:100DA0007C04C3EB13FBEA13FADCF7FFEB60027F72
:100DB000FFC23691CE2278A5E6F954037000E954BB
:100DC0000C7000E954307000E954C070002275675F
:100DD000007568007597DE7597AD7581C043FF801B
:100DE00075EF0675A90071BB75803F75F1C375A4D9
:100DF000C075803F75D4FF75900075F20F75A50F13
:100E000075900075D50F75A60175E34075E2027106
:100E1000BBE4F8F6D8FD71CE12145C789886647540
:100E20003001C2AF1205887150120580715612054B
:100E300080715C120580B1B6C2AF7567007568003D
:100E400078FA79FA308007D9FBD8F7021C00916054
:100E500091CE7898866471BB75A91375A71075C17A
:100E60000075A70075660075E400758811758E041D
:100E700075890975C80475910475D84075D90875C8
:100E8000F783759E0075960275DA4A75DB0075A8C2
:100E90002375E69075B801759B80759D0075D10C22
:100EA00075BCB975BB1075E88075B201120574D2B6
:100EB000AF753C00C230120588C231C232C233C2A3
:100EC00034755200755300752200120584C3E52263
:100ED000940A5002E19ED231752200120584C3E5C6
:100EE00022940A5002E19EC231D2327522001205CC
:100EF00084C3E522940A5002E19E75E4807588510E
:100F0000758E017589AA758C00758D00C2A9D2AB4A
:100F1000D2AA756B80756A14756E50C232D2347560
:100F2000220A120584756A10C3E522940A755200DC
:100F30007553004069758E0C756B00756A28756E67
:100F40002875220A120584756A20C3E522940A7561
:100F500052007553004047758E0C756B80756A148E
:100F6000756E1475220A120584756A10C3E5229401
:100F70000A755200755300402575E4007588117597
:100F80008E04758909D2A9C2ABC2AAC234D2337504
:100F90002200120584C3E522940A4002C1381205DA
:100FA00078203003020E38C2AF715071507150D2A8
:100FB000AF120588203403303A030210621205781C
:100FC000788CE6C394015003021062E530C39401AB
:100FD00050030210627567A57568F17F02D23691E1
:100FE000CE120584C2AFC23691CEC3E554947FD2EF
:100FF000AF406F120574C2AF7162D2AFDFDF120D66
:1010000083C3EF7897F6120588B1497F0AD236126A
:101010000CCE120584C2AFC236120CCEC3E5549476
:101020007FD2AF50E6120574C2AF120B5012057C8E
:10103000120B50D2AFDFD6120D83EF24037896F651
:10104000F87997E7C394234003985006E82423785F
:1010500097F612058891A3B178120584120CCE027E
:101060000E38756700756800120584C3E554940155
:101070004003020FB4C2AF120B62120B62120B627A
:10108000D2AF120588753000E4F537F5380537E53D
:1010900037F4703F0538789AE67819146012783280
:1010A00014600D787D14600878FA146003753800B8
:1010B000C3E53898401D120BBB12057415387537FF
:1010C0000078998664C2AF120B62D2AF78988664BA
:1010D00012058412057CE5237003020E38C3E55423
:1010E0009401500AC3E5529401501602108D120566
:1010F00084E5237003020E38755200755300021206
:10110000A3C3E55294017017C2AF120BBB78998646
:1011100064120B5078988664D2AF1205844195C34F
:10112000E55294027017C2AF120BBB789986641215
:101130000B5678988664D2AF1205844195C3E55268
:1011400094037017C2AF120BBB78998664120B5CC4
:1011500078988664D2AF1205844195C3E552940411
:101160007017C2AF120BBB78998664120B62789825
:101170008664D2AF1205844195C3E5529405701779
:10118000C2AF120BBB78998664120B6278988664A2
:10119000D2AF1205844195C3E55294077019C3E597
:1011A000539406500201DD7401303A0274037888CA
:1011B000F6C238C2394195C3E55294087019C3E5A7
:1011C000539406500201DD7402303A0274047888A8
:1011D000F6D238D2394195C3E55294097017C3E568
:1011E000539406500201DD303A0BC37888E694022E
:1011F000F6C23A4195C3E552940A7016C3E553947A
:1012000006500201DD203A0A7888E62402F6D23A36
:101210004195C3E55294147025C3E55394065002DA
:1012200001DDC2AF901A0B740093D2AF7888F61329
:10123000C238C2394002D2384002D2398057C3E5A1
:101240005294157038C3E5539406404FC2AF901ABC
:101250000B740093D2AFF8B801027402B8020274A2
:1012600001B803027404B8040274037888F613C248
:1012700038C2394002D2384002D2398018C3E55210
:10128000940C70117567A57568F1C3E55394064019
:101290000A91A3D2AF755200755300756700756847
:1012A0000001DDC2AF120BBBE4D2AFE4F55EF52462
:1012B000F525F53D755E081205741205DD30EDFD6E
:1012C000A8BDA9BEE97001F8885F1205E1755E0846
:1012D000C2AF120648855D5B855D5CD2AF75A71015
:1012E00075C13075A70075A903756601303A07C24C
:1012F00038303502D238D228753900120AEF120B75
:101300002012065712065E12065712065E12065784
:101310001208E31209E0120A2B12065E1208D3200B
:101320002C03120597302C031205C71209E0120A8C
:101330005C12065E1208E31209E0120A8D12065EC4
:101340001208D31209E0120ABE12065E1208E31256
:1013500009E0120AEF12065E1205DD1208D3120927
:10136000E0120B201205E112065E302827855D5B36
:1013700079187A0CC3E53999400EC228D2298A3BE4
:10138000855D5B855D5C800CC3E554940140030280
:101390001310811A30291F202B1CE53B147006C244
:1013A00029D22A6110F53B203A07C3E55494014045
:1013B000030213108064753C00203A0F78FA79A478
:1013C000E760027803C3E55598504FE523604B3042
:1013D0003A17203805203507800F303502800A2063
:1013E0002B07D22B855D5B614078F0302B05855D46
:1013F0005B7820C3E548985003021310302B1BC2C2
:101400002BC238303502D238D229753B12855D5B4C
:101410006110053CE5546002811D753C00C2AF12AD
:101420000BBB75240075250075A91375A71075C130
:101430000075A700756600D2AF120584120BBB7849
:10144000A4E6600CC286D287C290D291C292D29397
:10145000C3E53C94044003020E380188901A0D78CD
:101460002091DCE520B4550AA391DCE520B4AA0262
:1014700080137567A57568F1120BCE91A37567008F
:10148000756800801D901A0378807B0A91DCA308A0
:10149000DBFA901A0F788C7B1A91DCA308DBFA90A8
:1014A0001A2922C2AFB11F91FC901A00741091E169
:1014B000A3740791E1A3742191E1901A0378807BD2
:1014C0000A91E0A308DBFA901A0F788C7B1A91E05E
:1014D000A308DBFAB132B110901A2922E493F62264
:1014E000E6438F01538FFDFFC3E583941C40012227
:1014F000EF8567B78568B7F0538FFE22438F0243AD
:101500008F018567B78568B7901A0DF0538FFC225D
:10151000901A0D745591E1901A0E74AA91E1227AF5
:101520003079D07820901A4091DCE520F709A3DAD1
:10153000F7227A3079D0901A40E791E109A3DAF9DD
:10154000227C05120588DCFB22C2AF120B50120B65
:1015500056120B5C120B6212057C120B50120B56CA
:10156000120B5C120B6212057C120B50120B5612FE
:101570000B5C120B62D2AF22C2AF120B62120B5C79
:10158000120B56120B5012057C120B62120B5C12DE
:101590000B56120B5012057C120B62120B5C120BD5
:0715A00056120B50D2AF22DE
:1019FD00020DCE100721FFFFFFFFFFFF09FF01FFC3
:101A0D0055AA01FFFFFFFFFF03FFFFFF25D0285061
:0D1A1D0004FF02FF7AFF0701FFFF0000FF3A
:101A400023435F485F3030232020202020202020A7
:101A500023424C48454C492445464D3842323123B7
:101A60002020202020202020202020202020202076
:101C0000C2AFC2D37597DE7597AD7581C075A90057
:101C100043FF80752438752503B1DB7529A5752A26
:101C2000F143F10153A4FED28075D4FF75E3407DEA
:101C3000FA780379E67C10752200752300901DE880
:101C40007B06752498752501308002814820800824
:101C5000D8FBD9F9DCF781BA308008D8FBD9F9DC98
:101C6000F781BAB19BE493A3C39A6004DDC381BA40
:101C7000DBDBB18D600281317B08E493FAA3B16EA6
:101C8000DBF87A30B16E752200752300B18DEAFC65
:101C9000EBFDC3ED94FE400EB18D8A278B28ED300D
:101CA000E0048A828B83B18D7AC270D8C3ED94FE32
:101CB000601950CEBD0029EC600F7520007521FF22
:101CC000752900752A000200008100A827A92808AC
:101CD00009D804D90281DDB191EAF281D10D81A642
:101CE000C3ED94035051EDA2E092007AC5C3E582A2
:101CF0009400E583941C508C200010438F02438F86
:101D0000018529B7852AB7F0300027A827A9280818
:101D100009438F01538FFDD804D902A132C3E58353
:101D2000941C4003A3A117E28529B7852AB7F0A325
:101D3000A117538FFC81827AC1BD030CE493A3FAEF
:101D4000B152DCF8B14A81828184AA22AB23B16E00
:101D5000EBFAEA6222752608C3E52313F523E52290
:101D600013F52250066323A0632201D526EAB1DBD6
:101D7000B1DB75260AEAF4200102D280300102C2EA
:101D800080B1DBC3134002C201D526EB22B191EA38
:101D9000FB208002A191308002A196752608AE2416
:101DA000AF25C3EF13FFEE13FEB1DFB1DBC3EA13C0
:101DB0003080024480FA30E703632201C3E5231335
:101DC000F523E52213F52250066323A0632201D5F3
:101DD00026D9E52265236523F52222AE24AF250E00
:101DE0000FDEFEDFFCD20122424C48656C693437BD
:061DF0003164E8B20601B7
:00000001FF
